:020000040000FA
:0408000054EF09F0B8
:1008100003B283EF05F0F2B4A1EF05F09EB0A9EFAB
:1008200005F09EB2B1EF05F0F2A81AEF04F0F2B2B3
:1008300032EF04F09EB61FEF04F003EF09F09E962E
:1008400000011350000A06E000011350010A06E0FF
:1008500003EF09F0E8EC1CF003EF09F0DCEC1EF00C
:1008600003EF09F0CD90F2929EA03CEF04F001015D
:10087000533F3CEF04F0542BAEC1B2F1AFC1B3F122
:10088000B0C1B4F1B1C1B5F1AAC1AEF1ABC1AFF124
:10089000ACC1B0F1ADC1B1F1A6C1AAF1A7C1ABF134
:1008A000A8C1ACF1A9C1ADF1A2C1A6F1A3C1A7F144
:1008B000A4C1A8F1A5C1A9F19EC1A2F19FC1A3F154
:1008C000A0C1A4F1A1C1A5F19AC19EF19BC19FF164
:1008D0009CC1A0F19DC1A1F196C19AF197C19BF174
:1008E00098C19CF199C19DF1CECF96F1CFCF97F1F0
:1008F00053C198F154C199F1CF6ACE6A0101536B8B
:10090000546B9E90CD800FBC0F8E0FBA8BEF04F00E
:100910000F8A03EF09F00F8C0FBEC7EF04F096C1EA
:100920009AF197C19BF198C19CF199C19DF19AC12F
:100930009EF19BC19FF19CC1A0F19DC1A1F19EC1FF
:10094000A2F19FC1A3F1A0C1A4F1A1C1A5F1A2C1CF
:10095000A6F1A3C1A7F1A4C1A8F1A5C1A9F1A6C19F
:10096000AAF1A7C1ABF1A8C1ACF1A9C1ADF1AAC16F
:10097000AEF1ABC1AFF1ACC1B0F1ADC1B1F1AEC13F
:10098000B2F1AFC1B3F1B0C1B4F1B1C1B5F1010180
:100990005E6B5F6B606B616B96515E2797515F2357
:1009A00098516023995161239A515E279B515F238F
:1009B0009C5160239D5161239E515E279F515F236F
:1009C000A0516023A1516123A2515E27A3515F234F
:1009D000A4516023A5516123A6515E27A7515F232F
:1009E000A8516023A9516123AA515E27AB515F230F
:1009F000AC516023AD516123AE515E27AF515F23EF
:100A0000B0516023B1516123B2515E27B3515F23CE
:100A1000B4516023B5516123D89001016133603333
:100A20005F335E33D8900101613360335F335E33EF
:100A3000D8900101613360335F335E3300C10CF144
:100A400001C10DF102C10EF103C10FF104C110F19A
:100A500005C111F106C112F107C113F108C114F16A
:100A600009C115F10AC116F10BC117F134C135F1F5
:100A700011B846EF05F00101620E046F010E056F1B
:100A8000000E066F000E076F4FEF05F00101A70E75
:100A9000046F020E056F000E066F000E076F5EC139
:100AA00000F15FC101F160C102F161C103F17FECAE
:100AB0001BF003BF04D018BE02D018A0108C11A0E8
:100AC00067EF05F010BA67EF05F00F80108A0CC1D0
:100AD00000F10DC101F10EC102F10FC103F110C10E
:100AE00004F111C105F112C106F113C107F114C1DE
:100AF00008F115C109F116C10AF117C10BF135C191
:100B000034F103EF09F00392ABB2AB98AB88030169
:100B100003EE00F080517F0BE92604C0EFFF802B2D
:100B20008151805D700BD8A48B8200008051815D63
:100B3000700BD8A48B9281518019D8B4079003EF21
:100B400009F0F2940101453F03EF09F0462B03EF52
:100B500009F09E900101533F03EF09F0542B03EF7E
:100B600009F09E9211B819EF07F08BB4BFEF05F0B2
:100B700010ACBFEF05F08B84109CC0EF05F08B9498
:100B8000C3CF55F1C4CF56F1C28207B42AEF06F0A5
:100B900047C14BF148C14CF149C14DF14AC14EF139
:100BA0005EC162F15FC163F160C164F161C165F171
:100BB00096C1B6F197C1B7F198C1B8F199C1B9F131
:100BC0009AC1BAF19BC1BBF19CC1BCF19DC1BDF101
:100BD0009EC1BEF19FC1BFF1A0C1C0F1A1C1C1F1D1
:100BE000A2C1C2F1A3C1C3F1A4C1C4F1A5C1C5F1A1
:100BF000A6C1C6F1A7C1C7F1A8C1C8F1A9C1C9F171
:100C0000AAC1CAF1ABC1CBF1ACC1CCF1ADC1CDF140
:100C1000AEC1CEF1AFC1CFF1B0C1D0F1B1C1D1F110
:100C2000B2C1D2F1B3C1D3F1B4C1D4F1B5C1D5F1E0
:100C3000010155515B2756515C23E86A5D230E2E56
:100C40002AEF06F05CC157F15DC158F15B6B5C6B3C
:100C50005D6B078E0201002F03EF09F03C0E006F61
:100C600016AE108E00C10CF101C10DF102C10EF1E2
:100C700003C10FF104C110F105C111F106C112F158
:100C800007C113F108C114F109C115F10AC116F128
:100C90000BC117F134C135F101018A6757EF06F036
:100CA0008B6757EF06F08C6757EF06F08D675BEFA9
:100CB00006F08BEF06F08EC100F18FC101F190C1FB
:100CC00002F191C103F10101010E046F000E056FE5
:100CD000000E066F000E076F7FEC1BF000C18EF157
:100CE00001C18FF102C190F103C191F1006780EF62
:100CF00006F0016780EF06F0026780EF06F00367F9
:100D00008BEF06F08AC18EF18BC18FF18CC190F10F
:100D10008DC191F10F80D57ED5BE6DD0D6CF47F174
:100D2000D7CF48F145C149F1E86AE8CF4AF118BE8A
:100D300002D018A0108C109047C100F148C101F1F9
:100D400049C102F14AC103F101010A0E046F000E0C
:100D5000056F000E066F000E076F7FEC1BF003AFF0
:100D60001080010154A7C1EF06F00F9A0F9C0F9E4F
:100D70000101000E5E6F600E5F6F3D0E606F080E2A
:100D8000616F010147BFD1EF06F04867D1EF06F070
:100D90004967D1EF06F04A67D1EF06F0F288F6EF27
:100DA00006F0F2985E6B5F6B606B616B966B976B96
:100DB000986B996B9A6B9B6B9C6B9D6B9E6B9F6BFF
:100DC000A06BA16BA26BA36BA46BA56BA66BA76BAF
:100DD000A86BA96BAA6BAB6BAC6BAD6BAE6BAF6B5F
:100DE000B06BB16BB26BB36BB46BB56BD76AD66AD1
:100DF0000101456B466B0CC100F10DC101F10EC143
:100E000002F10FC103F110C104F111C105F112C1CA
:100E100006F113C107F114C108F115C109F116C19A
:100E20000AF117C10BF135C134F103EF09F003EFFB
:100E300009F00201002F6AEF08F0D59ED6CF47F1E6
:100E4000D7CF48F145C149F1E86AE8CF4AF1D76AFE
:100E5000D66A0101456B466BD58E108E16AE198C85
:100E600000C10CF101C10DF102C10EF103C10FF17E
:100E700004C110F105C111F106C112F107C113F14E
:100E800008C114F109C115F10AC116F10BC117F11E
:100E900034C135F10FA0109A11B85AEF07F00101D3
:100EA000620E046F010E056F000E066F000E076FD5
:100EB00063EF07F00101A70E046F020E056F000E2D
:100EC000066F000E076F47C100F148C101F149C12B
:100ED00002F14AC103F17FEC1BF003BF76EF07F08C
:100EE00018BE02D018A0108C11B00F800CC100F1F8
:100EF0000DC101F10EC102F10FC103F110C104F1E6
:100F000011C105F112C106F113C107F114C108F1B5
:100F100015C109F116C10AF117C10BF135C134F140
:100F200002013C0E006F00C10CF101C10DF102C1C4
:100F30000EF103C10FF104C110F105C111F106C199
:100F400012F107C113F108C114F109C115F10AC169
:100F500016F10BC117F134C135F101018A67B8EF01
:100F600007F08B67B8EF07F08C67B8EF07F08D6775
:100F7000BCEF07F0ECEF07F08EC100F18FC101F17B
:100F800090C102F191C103F10101010E046F000E45
:100F9000056F000E066F000E076F7FEC1BF000C19F
:100FA0008EF101C18FF102C190F103C191F100678F
:100FB000E1EF07F00167E1EF07F00267E1EF07F00B
:100FC0000367ECEF07F08AC18EF18BC18FF18CC102
:100FD00090F18DC191F10F80109047C100F148C18F
:100FE00001F149C102F14AC103F101010A0E046F86
:100FF000000E056F000E066F000E076F7FEC1BF0F2
:1010000003AF1080010154A712EF08F00F9A0F9C54
:101010000F9E0101000E5E6F600E5F6F3D0E606FF0
:10102000080E616F47C100F148C101F149C102F1E9
:101030004AC103F10101140E046F050E056F000E85
:10104000066F000E076F7FEC1BF003AF2BEF08F06D
:10105000F28850EF08F0F2985E6B5F6B606B616B2B
:10106000966B976B986B996B9A6B9B6B9C6B9D6B5C
:101070009E6B9F6BA06BA16BA26BA36BA46BA56B0C
:10108000A66BA76BA86BA96BAA6BAB6BAC6BAD6BBC
:10109000AE6BAF6BB06BB16BB26BB36BB46BB56B6C
:1010A0000CC100F10DC101F10EC102F10FC103F13C
:1010B00010C104F111C105F112C106F113C107F10C
:1010C00014C108F115C109F116C10AF117C10BF1DC
:1010D00035C134F19BEC1FF01A661ED019AE11D049
:1010E000199E1A8E17AE07D0136A040E146E156A75
:1010F000E8EC1CF011D0136A146A156AE8EC1CF0D5
:101100000BD019AC09D0199C1A8C010E136E146AFD
:10111000156ADCEC1EF000D08BB496EF08F010AC32
:1011200096EF08F08B84109C97EF08F08B94C3CF58
:1011300055F1C4CF56F1C28207B401EF09F047C19F
:101140004BF148C14CF149C14DF14AC14EF15EC16C
:1011500062F15FC163F160C164F161C165F196C183
:10116000B6F197C1B7F198C1B8F199C1B9F19AC177
:10117000BAF19BC1BBF19CC1BCF19DC1BDF19EC147
:10118000BEF19FC1BFF1A0C1C0F1A1C1C1F1A2C117
:10119000C2F1A3C1C3F1A4C1C4F1A5C1C5F1A6C1E7
:1011A000C6F1A7C1C7F1A8C1C8F1A9C1C9F1AAC1B7
:1011B000CAF1ABC1CBF1ACC1CCF1ADC1CDF1AEC187
:1011C000CEF1AFC1CFF1B0C1D0F1B1C1D1F1B2C157
:1011D000D2F1B3C1D3F1B4C1D4F1B5C1D5F101019C
:1011E00055515B2756515C23E86A5D230E2E01EFB3
:1011F00009F05CC157F15DC158F15B6B5C6B5D6BD5
:10120000078E03EF09F002C0E0FF005001C0D8FFD5
:101210001000A6B209EF09F00CC0A9FF0BC0A8FF8F
:10122000A69EA69CA684F29E550EA76EAA0EA76E39
:10123000A682F28EA694A6B21BEF09F00C2A120029
:10124000A96EA69EA69CA680A8500C2A1200040196
:101250002C0E826F18EC0BF07AEC1CF00C5020EC8A
:1012600009F0E8CF00F10C5020EC09F0E8CF01F1D3
:1012700001AF40EF09F00101FF0E026FFF0E036F97
:101280001DEC1CF029674CEF09F00401200E826F61
:1012900018EC0BF051EF09F004012D0E826F18ECE1
:1012A0000BF047EC1AF01200076A0F6A106A116A15
:1012B000126A0F010E0EC16E860EC06E030EC26E54
:1012C0000F01896A110E926E080E8A6EF10E936EEE
:1012D0008B6A980E946EF18EFC0E20EC09F0E8CF2C
:1012E0000BF00BA011800BA211820BA411840BA890
:1012F0001188C90E20EC09F0E8CF16F0CA0E20ECD8
:1013000009F0E8CF17F0CB0E20EC09F0E8CF18F089
:10131000196A1A6A0E6A01015B6B5C6B5D6B576B35
:10132000586BF29A0101476B486B496B4A6B4B6BE8
:101330004C6B4D6B4E6B4F6B506B516B526B456BE7
:10134000466BD76AD66A0F01280ED56EF28A9D9039
:10135000B00ECD6E01015E6B5F6B606B616B626B9B
:10136000636B646B656B666B676B686B696B536B08
:10137000546BCF6ACE6A0F9A0F9C0F9E9D80760E9B
:10138000CA6E9D8202013C0E006FCC6A160E20ECE4
:1013900009F0E8CF00F1170E20EC09F0E8CF01F1D9
:1013A000180E20EC09F0E8CF02F1190E20EC09F03C
:1013B000E8CF03F1010103AFF8EF09F07AEC1CF07C
:1013C000160E0C6E00C10BF009EC09F0170E0C6E36
:1013D00001C10BF009EC09F0180E0C6E02C10BF004
:1013E00009EC09F0190E0C6E03C10BF009EC09F0C1
:1013F00000C18AF101C18BF102C18CF103C18DF1F1
:1014000000C18EF101C18FF102C190F103C191F1D0
:101410001A0E20EC09F0E8CF00F11B0E20EC09F0C9
:10142000E8CF01F11C0E20EC09F0E8CF02F11D0E0F
:1014300020EC09F0E8CF03F1010103AF4EEF0AF011
:101440007AEC1CF01A0E0C6E00C10BF009EC09F0DE
:101450001B0E0C6E01C10BF009EC09F01C0E0C6E9A
:1014600002C10BF009EC09F01D0E0C6E03C10BF06C
:1014700009EC09F01A0E20EC09F0E8CF00F11B0E80
:1014800020EC09F0E8CF01F11C0E20EC09F0E8CFC8
:1014900002F11D0E20EC09F0E8CF03F100C192F13A
:1014A00001C193F102C194F103C195F1240EAC6E18
:1014B000900EAB6E240EAC6E080EB86E000EB06EC1
:1014C0001F0EAF6E0401806B816B0F01900EAB6E2F
:1014D0000F019D8A0301806B816BC26B8B92136A33
:1014E000146A156A9D8607900001F28EF28C07B08F
:1014F000F4EF18F00FB04DEF13F010BE4DEF13F0F6
:101500000301805181197F0BD8B4F4EF18F013EE6A
:1015100000F081517F0BE126812BE7CFE8FFE00B44
:10152000D8B4F4EF18F023EE82F0C2513F0BD92665
:10153000E7CFDFFFC22BDF50780AD8A4F4EF18F012
:1015400007808EC100F18FC101F190C102F191C1FC
:1015500003F10101040E046F000E056F000E066F0B
:10156000000E076F7FEC1BF000AFC0EF0AF0010127
:10157000030E8E6F000E8F6F000E906F000E916F36
:1015800003018251720AD8B44AEF13F08251520A11
:10159000D8B44AEF13F08251750AD8B44AEF13F069
:1015A0008251630AD8B4AEEF15F08251690AD8B4FB
:1015B000F1EF0FF082517A0AD8B404EF11F08251A2
:1015C000490AD8B490EF0FF08251500AD8B4A2EF74
:1015D0000EF08251700AD8B4E8EF0EF08251540A2E
:1015E000D8B416EF0FF08251740AD8B45FEF0FF041
:1015F0008251410AD8B42CEF0BF082516D0AD8B455
:10160000FAEF0DF082514D0AD8B413EF0EF082516B
:10161000730AD8B47AEF12F08251530AD8B4DFEFCC
:1016200012F08251590AD8B44BEF0DF0E5EF15F0E6
:10163000040114EE00F080517F0BE12682C4E7FF25
:10164000802B120004010D0E826F18EC0BF00A0EB5
:10165000826F18EC0BF012000401410E826F18EC3F
:101660000BF003018351310AD8B46BEF0CF0030186
:101670008351320AD8B4C1EF0BF003018351330A0E
:10168000D8B44AEF0BF004013F0E826F18EC0BF058
:10169000E3EF15F0CB0E20EC09F0E8CF0BF00401DE
:1016A0002C0E826F18EC0BF003018451450AD8B45C
:1016B0006EEF0BF003018451440AD8B471EF0BF0C4
:1016C00003018451300AD8B474EF0BF00301845144
:1016D000310AD8B478EF0BF083EF0BF00B9E7DEF5F
:1016E0000BF00B8E7DEF0BF0FC0E0B167DEF0BF06D
:1016F000FC0E0B160B807DEF0BF0CB0E0C6E0BC0AF
:101700000BF009EC09F00401330E826F18EC0BF0BA
:1017100004012C0E826F18EC0BF0CB0E20EC09F0BC
:10172000E8CF18F018BE9CEF0BF00401450E826F55
:1017300018EC0BF0A1EF0BF00401440E826F18ECD3
:101740000BF004012C0E826F18EC0BF00401300E2C
:10175000826F18EC0BF004012C0E826F18EC0BF06A
:1017600018B0BAEF0BF00401300E826F18EC0BF0DA
:10177000BFEF0BF00401310E826F18EC0BF0E3EFBA
:1017800015F0CA0E20EC09F0E8CF0BF004012C0E86
:10179000826F18EC0BF003018451450AD8B4F1EFC5
:1017A0000BF003018451440AD8B4F4EF0BF00301A9
:1017B00084514D0AD8B4FDEF0BF003018451410A66
:1017C000D8B4F7EF0BF003018451460AD8B4FAEF0E
:1017D0000BF003018451560AD8B405EF0CF016EF54
:1017E0000CF00B9E10EF0CF00B8E10EF0CF00B9C1E
:1017F00010EF0CF00B8C10EF0CF0F80E0B1685C3ED
:10180000E8FF070B0B1210EF0CF0C70E0B1685C389
:10181000E8FF070BE846E846E8460B1210EF0CF02D
:10182000CA0E0C6E0BC00BF009EC09F0CA0E20ECCE
:1018300009F0E8CF17F00401320E826F18EC0BF0BC
:1018400004012C0E826F18EC0BF017BE2FEF0CF07A
:101850000401450E826F18EC0BF034EF0CF004011C
:10186000440E826F18EC0BF004012C0E826F18EC02
:101870000BF017C0E8FF070BE8CF82F40401300E2D
:10188000822718EC0BF004012C0E826F18EC0BF081
:1018900017BC52EF0CF00401410E826F18EC0BF0F4
:1018A00057EF0CF00401460E826F18EC0BF00401A8
:1018B0002C0E826F18EC0BF017C0E8FF380BE842D3
:1018C000E842E842E8CF82F40401300E822718ECA7
:1018D0000BF0E3EF15F0C90E20EC09F0E8CF0BF0A8
:1018E00004012C0E826F18EC0BF003018451450AA1
:1018F000D8B489EF0CF003018451440AD8B48CEFBA
:101900000CF0030184514D0AD8B48FEF0CF09DEF19
:101910000CF00B9E97EF0CF00B8E97EF0CF0F80E7F
:101920000B1685C3E8FF070B0B1297EF0CF0C90EDF
:101930000C6E0BC00BF009EC09F00401310E826F44
:1019400018EC0BF004012C0E826F18EC0BF0C90E92
:1019500020EC09F0E8CF16F016BE06D00401450EC3
:10196000826F18EC0BF005D00401440E826F18EC66
:101970000BF004012C0E826F18EC0BF016C0E8FF80
:10198000070BE8CF82F40401300E822718EC0BF02D
:1019900004012C0E826F18EC0BF007807AEC1CF01F
:1019A00025C0E8FF003B00430043030B1DEC1CF087
:1019B00033C182F40401300E822718EC0BF00401CD
:1019C0002C0E826F18EC0BF07AEC1CF025C001F1A4
:1019D000019F019D26C000F101011DEC1CF02FC1EB
:1019E00082F40401300E822718EC0BF030C182F42F
:1019F0000401300E822718EC0BF031C182F404018F
:101A0000300E822718EC0BF032C182F40401300E44
:101A1000822718EC0BF033C182F40401300E8227C8
:101A200018EC0BF004012C0E826F18EC0BF07AEC22
:101A30001CF027C001F128C000F1D8900133003319
:101A4000D8900133003301011DEC1CF02FC182F44A
:101A50000401300E822718EC0BF030C182F404012F
:101A6000300E822718EC0BF031C182F40401300EE5
:101A7000822718EC0BF032C182F40401300E822769
:101A800018EC0BF033C182F40401300E822718ECFD
:101A90000BF0E3EF15F0FC0E20EC09F0E8CF0BF0B3
:101AA00003018351520AD8B482EF0DF00301835130
:101AB000720AD8B485EF0DF003018351500AD8B4EF
:101AC00088EF0DF003018351700AD8B48BEF0DF04D
:101AD00003018351550AD8B48EEF0DF003018351F1
:101AE000750AD8B491EF0DF003018351430AD8B4BD
:101AF0009AEF0DF003018351630AD8B49DEF0DF006
:101B0000A6EF0DF00B90A0EF0DF00B80A0EF0DF005
:101B10000B92A0EF0DF00B82A0EF0DF00B94A0EF55
:101B20000DF00B84A0EF0DF00B96A0EF0DF00B86DF
:101B3000A0EF0DF00B98A0EF0DF00B88A0EF0DF0CB
:101B4000FC0E0C6E0BC00BF009EC09F00401590EF1
:101B5000826F18EC0BF01190119211941198FC0EF9
:101B600020EC09F0E8CF0BF00BA011800BA2118242
:101B70000BA411840BA8118811A0C6EF0DF004016D
:101B8000520E826F18EC0BF0CBEF0DF00401720EC9
:101B9000826F18EC0BF011A8D5EF0DF00401430E85
:101BA000826F18EC0BF0DAEF0DF00401630E826F18
:101BB00018EC0BF011A2E4EF0DF00401500E826F4F
:101BC00018EC0BF0E9EF0DF00401700E826F18ECC9
:101BD0000BF011A4F3EF0DF00401550E826F18EC19
:101BE0000BF0F8EF0DF00401750E826F18EC0BF09E
:101BF000E3EF15F004016D0E826F18EC0BF003019A
:101C00008351300AD8B452EF0EF003018351310AE8
:101C1000D8B465EF0EF003018351320AD8B478EFDF
:101C20000EF0E5EF15F004014D0E826F18EC0BF08D
:101C3000BBEC1CF084C331F185C332F186C333F1B0
:101C40000101296BC8EC1CF03FEC1CF0030183512F
:101C5000300AD8B43AEF0EF003018351310AD8B4F8
:101C600042EF0EF003018351320AD8B44AEF0EF06E
:101C7000E5EF15F0FD0E0C6E00C10BF009EC09F05C
:101C800052EF0EF0FE0E0C6E00C10BF009EC09F0E5
:101C900065EF0EF0FF0E0C6E00C10BF009EC09F0C1
:101CA00078EF0EF00401300E826F18EC0BF0040197
:101CB0002C0E826F18EC0BF07AEC1CF0FD0E20EC71
:101CC00009F0E8CF00F189EF0EF00401310E826FC8
:101CD00018EC0BF004012C0E826F18EC0BF07AEC70
:101CE0001CF0FE0E20EC09F0E8CF00F189EF0EF0B9
:101CF0000401320E826F18EC0BF07AEC1CF0040138
:101D00002C0E826F18EC0BF0FF0E20EC09F0E8CFE0
:101D100000F11DEC1CF031C182F40401300E822769
:101D200018EC0BF032C182F40401300E822718EC5B
:101D30000BF033C182F40401300E822718EC0BF053
:101D4000E3EF15F081A890EF0FF083C32AF184C36D
:101D50002BF185C32CF186C32DF187C32EF188C3E7
:101D60002FF189C330F18AC331F18BC332F18CC3B7
:101D700033F10101C8EC1CF03FEC1CF0160E0C6EA8
:101D800000C10BF009EC09F0170E0C6E01C10BF04D
:101D900009EC09F0180E0C6E02C10BF009EC09F009
:101DA000190E0C6E03C10BF009EC09F000C18AF1A9
:101DB00001C18BF102C18CF103C18DF100C18EF123
:101DC00001C18FF102C190F103C191F190EF0FF0C9
:101DD00081A890EF0FF083C32AF184C32BF185C350
:101DE0002CF186C32DF187C32EF188C32FF189C34F
:101DF00030F18AC331F18BC332F18CC333F101016D
:101E0000C8EC1CF03FEC1CF000C18AF101C18BF161
:101E100002C18CF103C18DF100C18EF101C18FF1BE
:101E200002C190F103C191F190EF0FF081A890EF02
:101E30000FF083C32AF184C32BF185C32CF186C331
:101E40002DF187C32EF188C32FF189C330F18AC3E6
:101E500031F18CC332F18DC333F10101C8EC1CF0B8
:101E60003FEC1CF00101000E046F000E056F010E27
:101E7000066F000E076F90EC1BF01A0E0C6E00C17F
:101E80000BF009EC09F01B0E0C6E01C10BF009EC14
:101E900009F01C0E0C6E02C10BF009EC09F01D0ECE
:101EA0000C6E03C10BF009EC09F000C192F101C105
:101EB00093F102C194F103C195F190EF0FF081A865
:101EC00090EF0FF083C32AF184C32BF185C32CF16B
:101ED00086C32DF187C32EF188C32FF189C330F15A
:101EE0008AC331F18CC332F18DC333F10101C8ECE7
:101EF0001CF03FEC1CF00101000E046F000E056F9A
:101F0000010E066F000E076F90EC1BF000C192F1FE
:101F100001C193F102C194F103C195F190EF0FF06B
:101F2000160E20EC09F0E8CF00F1170E20EC09F0B6
:101F3000E8CF01F1180E20EC09F0E8CF02F1190EFC
:101F400020EC09F0E8CF03F11DEC1CF000EC1AF0D6
:101F50000401730E826F18EC0BF004012C0E826FDB
:101F600018EC0BF08AC100F18BC101F18CC102F1B8
:101F70008DC103F11DEC1CF000EC1AF00401730E8E
:101F8000826F18EC0BF004012C0E826F18EC0BF032
:101F90001A0E20EC09F0E8CF00F11B0E20EC09F03E
:101FA000E8CF01F11C0E20EC09F0E8CF02F11D0E84
:101FB00020EC09F0E8CF03F100EC16F004012C0E40
:101FC000826F18EC0BF092C100F193C101F194C142
:101FD00002F195C103F100EC16F022EC0BF0E5EFF5
:101FE00015F00401690E826F18EC0BF004012C0E41
:101FF000826F18EC0BF00101040E006F000E016FF0
:10200000000E026F000E036F1DEC1CF02CC182F459
:102010000401300E822718EC0BF02DC182F404016C
:10202000300E822718EC0BF02EC182F40401300E22
:10203000822718EC0BF02FC182F40401300E8227A6
:1020400018EC0BF030C182F40401300E822718EC3A
:102050000BF031C182F40401300E822718EC0BF032
:1020600032C182F40401300E822718EC0BF033C128
:1020700082F40401300E822718EC0BF004012C0EC0
:10208000826F18EC0BF00101030E006F000E016F60
:10209000000E026F000E036F1DEC1CF02CC182F4C9
:1020A0000401300E822718EC0BF02DC182F40401DC
:1020B000300E822718EC0BF02EC182F40401300E92
:1020C000822718EC0BF02FC182F40401300E822716
:1020D00018EC0BF030C182F40401300E822718ECAA
:1020E0000BF031C182F40401300E822718EC0BF0A2
:1020F00032C182F40401300E822718EC0BF033C198
:1021000082F40401300E822718EC0BF004012C0E2F
:10211000826F18EC0BF001012A0E006F000E016FA8
:10212000000E026F000E036F1DEC1CF02CC182F438
:102130000401300E822718EC0BF02DC182F404014B
:10214000300E822718EC0BF02EC182F40401300E01
:10215000822718EC0BF02FC182F40401300E822785
:1021600018EC0BF030C182F40401300E822718EC19
:102170000BF031C182F40401300E822718EC0BF011
:1021800032C182F40401300E822718EC0BF033C107
:1021900082F40401300E822718EC0BF004012C0E9F
:1021A000826F18EC0BF0200EF86EF76AF66A0401E5
:1021B0000900F5CF82F418EC0BF00900F5CF82F49A
:1021C00018EC0BF00900F5CF82F418EC0BF00900C5
:1021D000F5CF82F418EC0BF00900F5CF82F418EC7F
:1021E0000BF00900F5CF82F418EC0BF00900F5CFE5
:1021F00082F418EC0BF00900F5CF82F418EC0BF028
:1022000022EC0BF0E5EF15F08351630AD8A4E5EF5B
:1022100015F08451610AD8A4E5EF15F085516C0AD8
:10222000D8A4E5EF15F08651410A42E08651440AF0
:102230001BE08651420AD8B46BEF11F08651350A83
:10224000D8B46FEF17F08651360AD8B4C4EF17F040
:102250008651370AD8B42DEF18F08651380AD8B411
:102260008BEF18F0E5EF15F00798079A04017A0E46
:10227000826F18EC0BF00401780E826F18EC0BF0F3
:102280000401640E826F18EC0BF081A84FEF11F07F
:102290000401550E826F18EC0BF054EF11F004019D
:1022A0004C0E826F18EC0BF022EC0BF0E5EF15F002
:1022B0000788079A04017A0E826F18EC0BF004016C
:1022C000410E826F18EC0BF00401610E826F18EC66
:1022D0000BF045EF11F00798078A04017A0E826F20
:1022E00018EC0BF00401420E826F18EC0BF00401A5
:1022F000610E826F18EC0BF045EF11F0010166677B
:1023000089EF11F0676789EF11F0686789EF11F0C5
:102310006967A1EF11F04F6795EF11F0506795EFE6
:1023200011F0516795EF11F05267A1EF11F0010123
:10233000000E006F000E016F000E026F000E036FA3
:10234000120011B8AFEF11F00101620E046F010E1F
:10235000056F000E066F000E076FB8EF11F0010158
:10236000A70E046F020E056F000E066F000E076FBA
:1023700066C100F167C101F168C102F169C103F1F1
:102380007FEC1BF003BF36EF12F0119A0101000E33
:10239000046FA80E056F550E066F020E076F66C11B
:1023A00000F167C101F168C102F169C103F166C1C1
:1023B00086F167C187F168C188F169C189F17FEC55
:1023C0001BF003BFEFEF11F00101000E866FA80EA6
:1023D000876F550E886F020E896F118A119C0E0E41
:1023E00020EC09F0E8CF18F10F0E20EC09F0E8CF4F
:1023F00019F1100E20EC09F0E8CF1AF1110E20ECC3
:1024000009F0E8CF1BF1C8EC1AF086C104F187C1CE
:1024100005F188C106F189C107F17FEC1BF0078245
:102420008CEC1AF0C8EC1AF007928CEC1AF086C10A
:1024300000F187C101F188C102F189C103F107925E
:102440008CEC1AF0CC0E046FE00E056F870E066F51
:10245000050E076F7FEC1BF000C118F101C119F1E7
:1024600002C11AF103C11BF171EF12F0119C0101BD
:10247000800E006F1A0E016F060E026F000E036FC2
:102480004FC104F150C105F151C106F152C107F12C
:102490007FEC1BF003AF52EF12F07AEC1CF0118CC2
:1024A000119A12000E0E20EC09F0E8CF18F10F0E71
:1024B00020EC09F0E8CF19F1100E20EC09F0E8CF7C
:1024C0001AF1110E20EC09F0E8CF1BF14FC100F119
:1024D00050C101F151C102F152C103F107828CECEC
:1024E0001AF018C100F119C101F11AC102F11BC1A2
:1024F00003F112000401730E826F18EC0BF004015B
:102500002C0E826F18EC0BF0078462C166F163C178
:1025100067F164C168F165C169F14BC14FF14CC10C
:1025200050F14DC151F14EC152F157C159F158C14D
:102530005AF10794A0EC12F022EC0BF0E5EF15F045
:1025400066C100F167C101F168C102F169C103F11F
:1025500001011DEC1CF000EC1AF00401630E826F07
:1025600018EC0BF004012C0E826F18EC0BF04FC12D
:1025700000F150C101F151C102F152C103F1010159
:102580001DEC1CF000EC1AF00401660E826F18ECD2
:102590000BF004012C0E826F18EC0BF07AEC1CF09F
:1025A00059C100F15AC101F101011DEC1CF000EC10
:1025B0001AF00401740E826F18EC0BF012001082F6
:1025C0000401530E826F18EC0BF004012C0E826F85
:1025D00018EC0BF083C32AF184C32BF185C32CF1D3
:1025E00086C32DF187C32EF188C32FF189C330F143
:1025F0008AC331F18BC332F18CC333F10101C8ECD2
:102600001CF03FEC1CF000C166F101C167F102C192
:1026100068F103C169F18EC32AF18FC32BF190C316
:102620002CF191C32DF192C32EF193C32FF194C3DA
:1026300030F195C331F196C332F197C333F1010103
:10264000C8EC1CF03FEC1CF000C14FF101C150F18F
:1026500002C151F103C152F1BBEC1CF099C32FF13F
:102660009AC330F19BC331F19CC332F19DC333F166
:102670000101C8EC1CF03FEC1CF000C159F101C194
:102680005AF1A0EC12F004012C0E826F18EC0BF042
:1026900054EF13F018A001D0108C8251520A03E1BC
:1026A0000F8254EF13F00F928251750A03E11084E8
:1026B0005BEF13F0109411A062EF13F011A462EF1E
:1026C00013F010848251550A03E1108669EF13F06C
:1026D0001096078410B2C6EF13F010A4B2EF13F0F7
:1026E000B6C166F1B7C167F1B8C168F1B9C169F1A6
:1026F000BAC16AF1BBC16BF1BCC16CF1BDC16DF176
:10270000BEC16EF1BFC16FF1C0C170F1C1C171F145
:10271000C2C172F1C3C173F1C4C174F1C5C175F115
:10272000C6C176F1C7C177F1C8C178F1C9C179F1E5
:10273000CAC17AF1CBC17BF1CCC17CF1CDC17DF1B5
:10274000CEC17EF1CFC17FF1D0C180F1D1C181F185
:10275000D2C182F1D3C183F1D4C184F1D5C185F155
:10276000BAEF13F062C166F163C167F164C168F149
:1027700065C169F14BC14FF14CC150F14DC151F1EF
:102780004EC152F157C159F158C15AF107940FA0E7
:10279000E8EF13F001019267D5EF13F09367D5EFDF
:1027A00013F09467D5EF13F09567D9EF13F0E8EFC6
:1027B00013F07EEC11F092C104F193C105F194C1C4
:1027C00006F195C107F17FEC1BF003BFABEF15F0ED
:1027D0007EEC11F00101000E046F000E056F010E7A
:1027E000066F000E076FB0EC1BF011A027EF14F07E
:1027F00011A227EF14F01DEC1CF0296702EF14F072
:1028000009EF14F004012D0E826F18EC0BF0A9EF04
:1028100015F030C182F40401300E822718EC0BF061
:1028200031C182F40401300E822718EC0BF032C162
:1028300082F40401300E822718EC0BF033C182F4CD
:102840000401300E822718EC0BF0A9EF15F010AE42
:102850004BD0109E00C108F101C109F102C10AF17B
:1028600003C10BF11DEC1CF030C1D6F131C1D7F121
:1028700032C1D8F133C1D9F108C100F109C101F168
:102880000AC102F10BC103F101016C0E046F070EC6
:10289000056F000E066F000E076F7FEC1BF003BF85
:1028A00004D00101550EDA6F1CD008C100F109C136
:1028B00001F10AC102F10BC103F10101A40E046F81
:1028C000060E056F000E066F000E076F7FEC1BF003
:1028D00003BF04D001017F0EDA6F03D00101FF0EA8
:1028E000DA6F198EABEF15F010A47EEF14F004012F
:1028F000750E826F18EC0BF083EF14F00401720E6A
:10290000826F18EC0BF004012C0E826F18EC0BF0A8
:102910001DEC1CF0296792EF14F00401200E826F69
:1029200095EF14F004012D0E826F18EC0BF030C1FE
:1029300082F40401300E822718EC0BF031C182F4CE
:102940000401300E822718EC0BF004012E0E826F6A
:1029500018EC0BF032C182F40401300E822718EC1F
:102960000BF033C182F40401300E822718EC0BF017
:1029700004016D0E826F18EC0BF004012C0E826FB7
:1029800018EC0BF04FC100F150C101F151C102F13F
:1029900052C103F101011DEC1CF000EC1AF004011E
:1029A000480E826F18EC0BF004017A0E826F18EC5F
:1029B0000BF004012C0E826F18EC0BF066C100F1D5
:1029C00067C101F168C102F169C103F101011DECA8
:1029D0001CF000EC1AF00401630E826F18EC0BF08F
:1029E00004012C0E826F18EC0BF066C100F167C178
:1029F00001F168C102F169C103F101010A0E046F1E
:102A0000000E056F000E066F000E076F90EC1BF0B6
:102A1000000E046F120E056F000E066F000E076F9A
:102A2000B0EC1BF01DEC1CF02AC182F40401300E46
:102A3000822718EC0BF02BC182F40401300E8227A0
:102A400018EC0BF02CC182F40401300E822718EC34
:102A50000BF02DC182F40401300E822718EC0BF02C
:102A60002EC182F40401300E822718EC0BF02FC126
:102A700082F40401300E822718EC0BF030C182F48E
:102A80000401300E822718EC0BF004012E0E826F29
:102A900018EC0BF031C182F40401300E822718ECDF
:102AA0000BF032C182F40401300E822718EC0BF0D7
:102AB00033C182F40401300E822718EC0BF00401BC
:102AC000730E826F18EC0BF004012C0E826F18EC61
:102AD0000BF07AEC1CF059C100F15AC101F10FEC76
:102AE00017F00FB277EF15F00FA0A9EF15F0040162
:102AF0002C0E826F18EC0BF0200EF86EF76AF66A57
:102B000004010900F5CF82F418EC0BF00900F5CFB1
:102B100082F418EC0BF00900F5CF82F418EC0BF0FE
:102B20000900F5CF82F418EC0BF00900F5CF82F420
:102B300018EC0BF00900F5CF82F418EC0BF009004B
:102B4000F5CF82F418EC0BF00900F5CF82F418EC05
:102B50000BF022EC0BF00F90E5EF15F00401630E83
:102B6000826F18EC0BF004012C0E826F18EC0BF046
:102B7000EBEC15F004012C0E826F18EC0BF05EEC00
:102B800016F004012C0E826F18EC0BF0DAEC16F044
:102B900004012C0E826F18EC0BF00101F80E006F8F
:102BA000CD0E016F660E026F030E036F00EC16F080
:102BB00004012C0E826F18EC0BF0F0EC16F022ECF6
:102BC0000BF0E5EF15F022EC0BF00301C26B079060
:102BD0001092F4EF18F0D8900E0E20EC09F0E8CF28
:102BE00000F10F0E20EC09F0E8CF01F1100E20ECFF
:102BF00009F0E8CF02F1110E20EC09F0E8CF03F163
:102C00000101000E046F000E056F010E066F000E2D
:102C1000076FB0EC1BF01DEC1CF02AC182F404011C
:102C2000300E822718EC0BF02BC182F40401300E19
:102C3000822718EC0BF02CC182F40401300E82279D
:102C400018EC0BF02DC182F40401300E822718EC31
:102C50000BF02EC182F40401300E822718EC0BF029
:102C60002FC182F40401300E822718EC0BF030C122
:102C700082F40401300E822718EC0BF031C182F48B
:102C80000401300E822718EC0BF004012E0E826F27
:102C900018EC0BF032C182F40401300E822718ECDC
:102CA0000BF033C182F40401300E822718EC0BF0D4
:102CB00004016D0E826F18EC0BF01200120E20EC66
:102CC00009F0E8CF00F1130E20EC09F0E8CF01F194
:102CD000140E20EC09F0E8CF02F1150E20EC09F0FB
:102CE000E8CF03F101010A0E046F000E056F000E1C
:102CF000066F000E076F90EC1BF0000E046F120EB3
:102D0000056F000E066F000E076FB0EC1BF01DEC98
:102D10001CF02AC182F40401300E822718EC0BF05B
:102D20002BC182F40401300E822718EC0BF02CC169
:102D300082F40401300E822718EC0BF02DC182F4CE
:102D40000401300E822718EC0BF02EC182F404012E
:102D5000300E822718EC0BF02FC182F40401300EE4
:102D6000822718EC0BF030C182F40401300E822768
:102D700018EC0BF004012E0E826F18EC0BF031C131
:102D800082F40401300E822718EC0BF032C182F479
:102D90000401300E822718EC0BF033C182F40401D9
:102DA000300E822718EC0BF00401730E826F18ECC2
:102DB0000BF012000A0E20EC09F0E8CF00F10B0E28
:102DC00020EC09F0E8CF01F10C0E20EC09F0E8CF7F
:102DD00002F10D0E20EC09F0E8CF03F10FEF17F030
:102DE000060E20EC09F0E8CF00F1070E20EC09F008
:102DF000E8CF01F1080E20EC09F0E8CF02F1090E4E
:102E000020EC09F0E8CF03F10FEF17F001017AECA5
:102E10001CF0078457C100F158C101F1079401016A
:102E2000E80E046F800E056F000E066F000E076F30
:102E300090EC1BF0000E046F040E056F000E066F81
:102E4000000E076FB0EC1BF0880E046F130E056FB9
:102E5000000E066F000E076F7FEC1BF00A0E046F6A
:102E6000000E056F000E066F000E076FB0EC1BF032
:102E70001DEC1CF00101296743EF17F00401200E3F
:102E8000826F46EF17F004012D0E826F18EC0BF0E5
:102E900030C182F40401300E822718EC0BF031C1EE
:102EA00082F40401300E822718EC0BF032C182F458
:102EB0000401300E822718EC0BF004012E0E826FF5
:102EC00018EC0BF033C182F40401300E822718ECA9
:102ED0000BF00401430E826F18EC0BF0120087C355
:102EE0002AF188C32BF189C32CF18AC32DF18BC33E
:102EF0002EF18CC32FF18DC330F18EC331F190C30D
:102F000032F191C333F10101296BC8EC1CF03FECA5
:102F10001CF00101000E046F000E056F010E066F1C
:102F2000000E076F90EC1BF00E0E0C6E00C10BF044
:102F300009EC09F00F0E0C6E01C10BF009EC09F061
:102F4000100E0C6E02C10BF009EC09F0110E0C6EA4
:102F500003C10BF009EC09F004017A0E826F18EC42
:102F60000BF004012C0E826F18EC0BF00401350EEF
:102F7000826F18EC0BF004012C0E826F18EC0BF032
:102F8000EBEC15F054EF11F087C32AF188C32BF155
:102F900089C32CF18AC32DF18BC32EF18CC32FF181
:102FA0008DC330F18EC331F190C332F191C333F14F
:102FB0000101296BC8EC1CF03FEC1CF0880E046F7B
:102FC000130E056F000E066F000E076F84EC1BF0EA
:102FD000000E046F040E056F000E066F000E076FE3
:102FE00090EC1BF00101E80E046F800E056F000EDF
:102FF000066F000E076FB0EC1BF00A0E0C6E00C1DE
:103000000BF009EC09F00B0E0C6E01C10BF009EC92
:1030100009F00C0E0C6E02C10BF009EC09F00D0E5C
:103020000C6E03C10BF009EC09F004017A0E826FFB
:1030300018EC0BF004012C0E826F18EC0BF004015D
:10304000360E826F18EC0BF004012C0E826F18EC18
:103050000BF0DAEC16F054EF11F087C32AF188C3B5
:103060002BF189C32CF18AC32DF18BC32EF18CC3B4
:103070002FF18DC330F18FC331F190C332F191C381
:1030800033F10101C8EC1CF03FEC1CF0000E046FA2
:10309000120E056F000E066F000E076F90EC1BF00E
:1030A00001010A0E046F000E056F000E066F000E80
:1030B000076FB0EC1BF0120E0C6E00C10BF009ECA8
:1030C00009F0130E0C6E01C10BF009EC09F0140E9F
:1030D0000C6E02C10BF009EC09F0150E0C6E03C169
:1030E0000BF009EC09F004017A0E826F18EC0BF07A
:1030F00004012C0E826F18EC0BF00401370E826F66
:1031000018EC0BF004012C0E826F18EC0BF05EEC47
:1031100016F054EF11F087C32AF188C32BF189C34D
:103120002CF18AC32DF18BC32EF18CC32FF18DC3EB
:1031300030F18EC331F190C332F191C333F101010B
:10314000296BC8EC1CF03FEC1CF0880E046F130ECA
:10315000056F000E066F000E076F84EC1BF0000E6B
:10316000046F040E056F000E066F000E076F90ECE3
:103170001BF00101E80E046F800E056F000E066F54
:10318000000E076FB0EC1BF0060E0C6E00C10BF0CA
:1031900009EC09F0070E0C6E01C10BF009EC09F007
:1031A000080E0C6E02C10BF009EC09F0090E0C6E52
:1031B00003C10BF009EC09F004017A0E826F18ECE0
:1031C0000BF004012C0E826F18EC0BF00401380E8A
:1031D000826F18EC0BF004012C0E826F18EC0BF0D0
:1031E000F0EC16F054EF11F081A8B2EF19F007A837
:1031F0006BEF19F00101800E006F1A0E016F060EC1
:10320000026F000E036F4BC104F14CC105F14DC1BB
:1032100006F14EC107F17FEC1BF003BFB2EF19F0CE
:10322000FAEC19F04BC100F14CC101F14DC102F1B2
:103230004EC103F107828CEC1AF018C104F119C1D8
:1032400005F11AC106F11BC107F1F80E006FCD0E92
:10325000016F660E026F030E036F7FEC1BF00E0E04
:103260000C6E00C10BF009EC09F00F0E0C6E01C1E1
:103270000BF009EC09F0100E0C6E02C10BF009EC1A
:1032800009F0110E0C6E03C10BF009EC09F0078474
:1032900001017AEC1CF057C100F158C101F107940B
:1032A0000A0E0C6E00C10BF009EC09F00B0E0C6E4F
:1032B00001C10BF009EC09F00C0E0C6E02C10BF011
:1032C00009EC09F00D0E0C6E03C10BF009EC09F0CE
:1032D0000798B2EF19F007AAB2EF19F007840101BD
:1032E0007AEC1CF057C100F158C101F10794060EA9
:1032F0000C6E00C10BF009EC09F0070E0C6E01C159
:103300000BF009EC09F0080E0C6E02C10BF009EC91
:1033100009F0090E0C6E03C10BF009EC09F00784EB
:1033200062C100F163C101F164C102F165C103F141
:103330000794120E0C6E00C10BF009EC09F0130E8D
:103340000C6E01C10BF009EC09F0140E0C6E02C1F9
:103350000BF009EC09F0150E0C6E03C10BF009EC33
:1033600009F0079A0401805181197F0B0BE09EA898
:1033700009D014EE00F081517F0BE126E750812B3C
:103380000F01AD6E77EF0AF018C100F119C101F11C
:103390001AC102F11BC103F1000E046F000E056F8C
:1033A000010E066F000E076FB0EC1BF029A1EFEFC6
:1033B00019F02051D8B4EFEF19F018C100F119C17C
:1033C00001F11AC102F11BC103F1000E046F000EDE
:1033D000056F0A0E066F000E076FB0EC1BF01200AF
:1033E0000101045100130551011306510213075145
:1033F000031312000101186B196B1A6B1B6B12007F
:103400002AC182F40401300E822718EC0BF02BC184
:1034100082F40401300E822718EC0BF02CC182F4E8
:103420000401300E822718EC0BF02DC182F4040148
:10343000300E822718EC0BF02EC182F40401300EFE
:10344000822718EC0BF02FC182F40401300E822782
:1034500018EC0BF030C182F40401300E822718EC16
:103460000BF031C182F40401300E822718EC0BF00E
:1034700032C182F40401300E822718EC0BF033C104
:1034800082F40401300E822718EC0BF012002FC1D9
:1034900082F40401300E822718EC0BF030C182F464
:1034A0000401300E822718EC0BF031C182F40401C4
:1034B000300E822718EC0BF032C182F40401300E7A
:1034C000822718EC0BF033C182F40401300E8227FE
:1034D00018EC0BF01200060E1B6E060E1C6E060E8C
:1034E0001D6E1B2E71EF1AF01C2E71EF1AF01D2E9F
:1034F00071EF1AF08B84020E1B6E020E1C6E020E10
:103500001D6E1B2E81EF1AF01C2E81EF1AF01D2E5E
:1035100081EF1AF08B9412000101005305E1015371
:1035200003E1025301E1002B4FEC1BF07AEC1CF09D
:103530003951006F3A51016F420E046F4B0E056F07
:10354000000E066F000E076F90EC1BF000C104F137
:1035500001C105F102C106F103C107F118C100F173
:1035600019C101F11AC102F11BC103F107B2BDEF8C
:103570001AF084EC1BF0BFEF1AF07FEC1BF000C1D7
:1035800018F101C119F102C11AF103C11BF11200B6
:103590007AEC1CF059C100F15AC101F1060E20EC81
:1035A00009F0E8CF04F1070E20EC09F0E8CF05F1AF
:1035B000080E20EC09F0E8CF06F1090E20EC09F026
:1035C000E8CF07F17FEC1BF000C124F101C125F128
:1035D00002C126F103C127F1290E046F000E056F09
:1035E000000E066F000E076F90EC1BF0EE0E046FDE
:1035F000430E056F000E066F000E076F84EC1BF084
:1036000024C104F125C105F126C106F127C107F146
:1036100090EC1BF000C11CF101C11DF102C11EF1B3
:1036200003C11FF1120E20EC09F0E8CF04F1130ED4
:1036300020EC09F0E8CF05F1140E20EC09F0E8CFFA
:1036400006F1150E20EC09F0E8CF07F10D0E006F22
:10365000000E016F000E026F000E036F90EC1BF066
:10366000180E046F000E056F000E066F000E076F38
:10367000B0EC1BF01CC104F11DC105F11EC106F127
:103680001FC107F184EC1BF06A0E046F2A0E056F50
:10369000000E066F000E076F7FEC1BF01200BF0ECE
:1036A000FA6E200E3A6F396BD89000370137023727
:1036B0000337D8B060EF1BF03A2F55EF1BF03907F6
:1036C0003A070353D8B412000331070B80093F6F48
:1036D00003390F0B010F396F80EC5FF0406F390534
:1036E00080EC5FF0405D405F396B3F33D8B03927E5
:1036F00039333FA975EF1BF0405139271200010102
:103700009FEC1CF0D8B01200010103510719346F6F
:1037100062EC1CF0D8900751031934AF800F1200EF
:103720000101346B86EC1CF0D8A09CEC1CF0D8B0E6
:10373000120071EC1CF07AEC1CF01F0E366FB2EC2C
:103740001CF00B35D8B062EC1CF0D8A00335D8B013
:103750001200362F9FEF1BF034B189EC1CF01200E1
:103760000101346B04510511061107110008D8A09E
:1037700086EC1CF0D8A09CEC1CF0D8B01200086BB2
:10378000096B0A6B0B6BB2EC1CF01F0E366FB2ECC0
:103790001CF007510B5DD8A4DAEF1BF006510A5D4F
:1037A000D8A4DAEF1BF00551095DD8A4DAEF1BF0BD
:1037B0000451085DD8A0EDEF1BF00451085F0551DE
:1037C000D8A0053D095F0651D8A0063D0A5F075104
:1037D000D8A0073D0B5FD8900081362FC7EF1BF0B4
:1037E00034B189EC1CF0346B86EC1CF0D890B6EC4C
:1037F0001CF007510B5DD8A40AEF1CF006510A5DBE
:10380000D8A40AEF1CF00551095DD8A40AEF1CF0FA
:103810000451085DD8A019EF1CF0003F19EF1CF00F
:10382000013F19EF1CF0023F19EF1CF0032BD8B435
:10383000120034B189EC1CF012000101346B86ECEB
:103840001CF0D8B01200BBEC1CF0200E366F003715
:1038500001370237033711EE33F00A0E376FE736C0
:103860000A0EE75CD8B0E76EE552372F2FEF1CF059
:10387000362F27EF1CF034B12981D89012000101B6
:103880000A0E346F200E366F11EE29F03451376F67
:103890000A0ED890E652D8B0E726E732372F4AEF23
:1038A0001CF00333023301330033362F44EF1CF096
:1038B000E750FF0FD8A00335D8B0120029B189EC2A
:1038C0001CF01200045100270551D8B0053D012716
:1038D0000651D8B0063D02270751D8B0073D03274F
:1038E00012000051086F0151096F02510A6F035114
:1038F0000B6F12000101006B016B026B036B120076
:103900000101046B056B066B076B12000335D8A031
:1039100012000351800B001F011F021F031F003FF5
:1039200099EF1CF0013F99EF1CF0023F99EF1CF05A
:10393000032B342B032512000735D8A012000751A2
:10394000800B041F051F061F071F043FAFEF1CF06D
:10395000053FAFEF1CF0063FAFEF1CF0072B342BF9
:1039600007251200003701370237033708370937B8
:103970000A370B3712000101296B2A6B2B6B2C6B5A
:103980002D6B2E6B2F6B306B316B326B336B1200E8
:1039900001012A510F0B2A6F2B510F0B2B6F2C514A
:1039A0000F0B2C6F2D510F0B2D6F2E510F0B2E6FF8
:1039B0002F510F0B2F6F30510F0B306F31510F0BF9
:1039C000316F32510F0B326F33510F0B336F1200C7
:1039D00000011550FF0A01E11200390EC86E800E79
:1039E000C76E280EC66E000EC56E1450000AD8B4FD
:1039F00023EF1DF01450010AD8B43CEF1DF0145011
:103A0000020AD8B455EF1DF01450030AD8B46EEF73
:103A10001DF01450040AD8B496EF1DF01450050A96
:103A2000D8B4AFEF1DF01450060AD8B4C8EF1DF09B
:103A30001450070AD8B4E1EF1DF01450080AD8B4A6
:103A4000FAEF1DF012001550000AD8B419EF1EF05D
:103A50001550010AD8B41DEF1EF01550020AD8B453
:103A600021EF1EF01550030AD8B425EF1EF01550B3
:103A7000040AD8B494EF1EF01550000AD8B429EF08
:103A80001EF01550010AD8B42DEF1EF01550020A91
:103A9000D8B431EF1EF01550030AD8B435EF1EF03C
:103AA0001550040AD8B494EF1EF01550000AD8B48B
:103AB00039EF1EF01550010AD8B43DEF1EF0155035
:103AC000020AD8B441EF1EF01550030AD8B445EFEE
:103AD0001EF01550040AD8B494EF1EF01550000AD9
:103AE000D8B452EF1EF01550010AD8B456EF1EF0AC
:103AF0001550020AD8B45AEF1EF01550030AD8B474
:103B00006EEF1EF01550040AD8B472EF1EF0155077
:103B1000050AD8B476EF1EF01550060AD8B47AEF2D
:103B20001EF01550070AD8B47DEF1EF01550000A9C
:103B3000D8B481EF1EF01550010AD8B485EF1EF0FD
:103B40001550020AD8B489EF1EF01550030AD8B4F4
:103B50008DEF1EF01550040AD8B490EF1EF01550EA
:103B6000000AD8B498EF1EF01550010AD8B49CEFA3
:103B70001EF01550020AD8B4A0EF1EF01550030A2B
:103B8000D8B4A4EF1EF01550040AD8B494EF1EF078
:103B90001550000AD8B4AEEF1EF01550010AD8B483
:103BA000B2EF1EF01550020AD8B4B6EF1EF0155051
:103BB000030AD8B4BAEF1EF01550040AD8B494EF33
:103BC0001EF01550000AD8B4BBEF1EF01550010AC4
:103BD000D8B4BFEF1EF01550020AD8B4C3EF1EF0E0
:103BE0001550030AD8B4C7EF1EF01550040AD8B414
:103BF00094EF1EF01550000AD8B4C8EF1EF015500F
:103C0000010AD8B4CCEF1EF01550020AD8B4D0EF98
:103C10001EF01550030AD8B4D4EF1EF01550040A54
:103C2000D8B4D5EF1EF01550050AD8B4D8EF1EF061
:103C300012009E96C580152A1200E20EC96E152A42
:103C40001200770EC96E152A1200020EC96E152ACF
:103C500012009E96C580152A1200E20EC96E152A22
:103C60001200790EC96E152A1200000EC96E152AAF
:103C700012009E96C580152A1200E20EC96E152A02
:103C800012007A0EC96E152A120017BC03D0DAC1D1
:103C9000E8FF04D01750E844E8441F09E8CFC9FF03
:103CA000152A12009E96C580152A1200E20EC96ED2
:103CB000152A120011BA03D011BC01D003D0050E91
:103CC000146E3ED00101D6676AEF1EF0100EC96E69
:103CD0006CEF1EF0D6C1C9FF152A1200D7C1C9FF6B
:103CE000152A1200D8C1C9FF152A1200D9C1C9FF6F
:103CF000152A1200C584152A1200FF0E156E1A9E91
:103D000012009E96C580152A1200E20EC96E152A71
:103D10001200760EC96E152A1200C584152A1200EB
:103D2000FF0E156E1A9E1200C584142A156A120021
:103D30009E96C580152A1200E20EC96E152A120041
:103D40007B0EC96E152A120011AA04D0230EC96E6B
:103D5000152A12001C0EC96E152A12009E96C580E7
:103D6000152A1200E20EC96E152A12007C0EC96EC9
:103D7000152A1200E9D79E96C580152A1200E20E78
:103D8000C96E152A12007D0EC96E152A1200DCD7E5
:103D90009E96C580152A1200E20EC96E152A1200E1
:103DA0007E0EC96E152A1200CFD7C584152A1200BF
:103DB000FF0E156E1A9E12001550FF0AD8B49AEF26
:103DC0001FF0390EC86E800EC76E280EC66E000E2C
:103DD000C56E1450000AD8B4F5EF1EF01450010A55
:103DE000D8B409EF1FF09AEF1FF01550000AD8B4AD
:103DF00047EF1FF01550010AD8B44BEF1FF01550D4
:103E0000020AD8B455EF1FF01550030AD8B458EF82
:103E10001FF01550000AD8B45EEF1FF01550010ACC
:103E2000D8B462EF1FF01550020AD8B46CEF1FF03F
:103E30001550030AD8B46FEF1FF01550040AD8B418
:103E400075EF1FF01550050AD8B478EF1FF0155024
:103E5000060AD8B47EEF1FF01550070AD8B481EFD8
:103E60001FF01550080AD8B487EF1FF01550090A43
:103E7000D8B48AEF1FF015500A0AD8B490EF1FF09B
:103E800015500B0AD8B493EF1FF09AEF1FF09E96CF
:103E9000C58099EF1FF016B004D04E0EC96E99EF91
:103EA0001FF0500EC96E99EF1FF0C58499EF1FF0F7
:103EB000142AFF0E156E12809AEF1FF09E96C58091
:103EC00099EF1FF016B004D04F0EC96E99EF1FF096
:103ED000510EC96E99EF1FF0C58699EF1FF0C9CF3B
:103EE00021F0C59AC58899EF1FF0C58699EF1FF09C
:103EF000C9CF22F0C59AC58899EF1FF0C58699EF02
:103F00001FF0C9CF23F0C59AC58899EF1FF0C58669
:103F100099EF1FF0C9CF24F0C58AC58899EF1FF02B
:103F2000C58499EF1FF0FF0E156E12861A9C9AEF4A
:103F30001FF0152A120012B012D012B213D012B410
:103F400014D012A6120007B01200129621C025F05C
:103F500022C026F023C027F024C028F012001290BF
:103F60001282120012921284120000011550FF0AF0
:0C3F700004E11294156ADCEC1EF0120053
:10BF0000E844F926000C160C2B0C3F0C520C640C68
:10BF1000760C860C960CA50CB30CC10CCF0CDC0C6B
:06BF2000E80CF40C000C1B
:00000001FF
